:030000000208A44F
:080003000280038E828F83222C
:08000B0002800BAE82AF8322DC
:08001300028013742D0173003B
:08001B0002801B11730171004A
:08002300028023111601710097
:03002B0002802B25
:10002E00217601730167216521872194018A01CE12
:10003E0021CE21A802091E020B3D017D0201BB0249
:10004E000A86020A8C020ACA02086502082B0207F7
:10005E00B602078C020A05214A3098FDC298E5992E
:10006E0022117174203099FDC299F59922117DC02B
:10007E00E0740D1173740A1173D0E022C2D51162AF
:10008E0031A8B41B03D3E422B40D05D2D5C3E422A8
:10009E00FA314A40E9CA1173116231A8B41B0280C9
:1000AE00E4B40D03EAC322B40804117380D0B4156E
:1000BE000280F7FB314A40E0CB1173EAC44BC322F6
:1000CE007A007B007C04C2D5116231A8B41B07D321
:1000DE00E4F583F58222B408028003B47F0CBC04DD
:1000EE000280E5117331390C80DEB40D108B838ADA
:1000FE0082BC0407E4F583F582D2D5C322FD314AD2
:10010E0040C6CD120073EDC0E03128D0E02AFAE4EB
:10011E003BFBDCB4C38A828B8322EBC454F0FBEA34
:10012E00C4540F4BFBEAC454F0FA22EAC4540FFA3B
:10013E00EBC454F04AFAEBC4540FFB22C324D05044
:10014E001424F64004240AC32224F9500824FA4049
:10015E00042410C322D322C0E0C4540F24F650024C
:10016E002407243A1173D0E0C0E0540F24F6500255
:10017E002407243A1173D0E022C0E0E5833165E50F
:10018E00823165D0E022C0E0E493A3600AA2E75476
:10019E007F1173400280F1D0E022C0E0C394614031
:1001AE0009941A5005D0E024E022D0E0227800C055
:1001BE00E0E4936008A2E7084003A380F4D0E022B5
:1001CE00C0E0C3309808E599B41B01D3C298D0E0C3
:1001DE0022900DD91145EF3165EE316531941162E2
:1001EE0031A875F0DFC0F075F001C0F0F5F0901099
:1001FE0000F18C5024758204E493B4FE150582E45C
:10020E0093B5F00E11717582203194117D75824077
:10021E00E4730583E583B400D8E5F0B43F07900F8F
:10022E00411145A1D0B44D07900F49114581C0B47D
:10023E005207900F4E1145A137B44407900F52113B
:10024E004541A8B45507900F551145C145B44E0709
:10025E00900F581145E137B44A07900F5C11458154
:10026E0012B44807900F6211458149B44507900FAB
:10027E006E1145818AB44307900F731145E113B493
:10028E005A0B74006012900F771145E147B449087C
:10029E00900F68114502076D017D900E7311457820
:1002AE00107A10760008DAFB1167B41B028072B464
:1002BE003A0679007141800A314A40EC7906714163
:1002CE0080E6742E11737C007160F87160F5837195
:1002DE0060F5827160B40102802D7022E8601471A5
:1002EE0060FA79017141EA120865E43402F971414C
:1002FE00A3D8E97160EC60B07904714180AAE8601E
:10030E00F27160D8FC80ECE860047160D8F3716023
:10031E00EC70E57138900E92114530987A11678025
:10032E00767138900E8A1145806D78007900D9FE6D
:10033E00D8FA22E95407232410F907E770020907B7
:10034E0022D3878209878309E5827005E5837001D0
:10035E00C322116731A8B41B06D0E0D0E080C2B42E
:10036E003A0A79057141D0E0D0E041D0314A5006C9
:10037E007907714180DCFA116731A8B41B0280D96C
:10038E00B43A0280DD314A50067907714180E8CADD
:10039E00C44AFA2CFCEA22EEC0E0EFC0E0900E99BF
:1003AE00114579107EA27F0E910E7EA87F0E910EC2
:1003BE007EAD7F0E910E7A05714F4009DAFA900EDE
:1003CE00E911458025900EB8114579167EBC7F0E39
:1003DE0091007ECD7F0E91007ED57F0E91007EDB4B
:1003EE007F0E91007EE07F0E9100D0E0FFD0E0FE08
:1003FE00017D714F50091171120ACA110611452261
:10040E00714F80F2900E1B114511063187900DE948
:10041E00114511CE20D5065002E10E110E117D9020
:10042E000EF711451106E4F5D0F5F0F8F9FAFBFCDC
:10043E00FDFEFF758108C0E0C0E0737A10117B11DC
:10044E00063187743A111E7B101106E493A33165B1
:10045E001171DBF7116F7B101106E493A3547FB477
:10046E007F01E424E04001E424201173DBEC117DD4
:10047E00D1CA110E31CE4002DAC5017D900E5D114A
:10048E004511063187743A111E74281173110EE44A
:10049E00933165900E361145118A20D510400E11FC
:1004AE0006120865117D1106A3110E8191900E683A
:1004BE000145900E25114578151171D8FC11457521
:1004CE008310F18C4002017D116F7582203194757D
:1004DE00822031BB7421C398F874201173D8FC7537
:1004EE0082003187780674201173D8FC758204E47B
:1004FE0093AA83B4FE05900F2F8018B4FD05900FBC
:10050E00368010B42305900F338008B4F90280EEC4
:10051E00900F3D11458A83117D74FFB5830281D4FE
:10052E000583E583B4009B81D4117B7AFF90100084
:10053E0015830583E583B400028021F18C501D756F
:10054E008204E4934403F460E9116F0A74412A11A2
:10055E001E11267582203194117DA140BAFF05909F
:10056E000DF20145900DE41145744111731116748D
:10057E00412A1173900DE911451162B41B02017DE0
:10058E00FB741FC39AEB400231A81173FB117DEB74
:10059E00C3944140CFFBEAC39B40C90B901000159A
:1005AE00830583E583B400028017F18C50137582A6
:1005BE0004E4934403F460E9DBE7117D7582408126
:1005CE003422900F1711457C3F900F44D13A7C4D49
:1005DE00D13A7C52D13A7C44D13A7C55D13A7C4EB8
:1005EE00D13A7C4AD13A7C48D13A7C49D13A7C45C1
:1005FE00D13A7C43D13A740060047C5AD13A900FC0
:10060E00251145901000F18C5020758204E493B4AE
:10061E00FE11116F0582E49311731126758220313C
:10062E0094117D0583E583B400DC017D116FEC111F
:10063E007311261145017DD1DC900F011145EB316F
:10064E0065EA31651145ED3165EC3165117D8D83BE
:10065E008C82A3AC82AD83900E1111451167B41B31
:10066E0002E10C117D8A828B83ECC39582FAED95A3
:10067E00837009EA603254F0700280027A10743A84
:10068E001173EA31653187E58325822AFBE43165F2
:10069E00E49331652BFBA3DAF7EBF4043165117D9E
:1006AE00D1CA31CE50C38056743A1173E4316531DC
:1006BE0065316504316574FF3165017BE8C0E07812
:1006CE000CE58C04000070FBD8F7D0E0F822117B0B
:1006DE00900E3F114511CE402120D51EC083C08201
:1006EE00117D900E49114511CEAD83AC82D0E0FA4A
:1006FE00D0E0FB400520D502017DD0E0D0E0117D99
:10070E00900DD10145D1DC900E531145116231A8E7
:10071E00B459EB117B8B838A82E4120865EDB583A5
:10072E0005ECB5820122A380F0900E08114511CE82
:10073E0040CE20D5CB110E017B117B900F7711454A
:10074E00742C111E900E531145116231A8B459AE7E
:10075E00117B1207B6900F7C5003900F8301451149
:10076E007D7800117DB88002017DE83165743A1103
:10077E00731171E6316508E8540F70F580E57582E6
:10078E0000E493B4A517A3E493B4E511A3E493B4E2
:10079E00E00BA3E493B4A505758200D32274FFB5D4
:1007AE008302C322058380D674006038908000E4F3
:1007BE0093F4700DA37400B582F57400B583F0C385
:1007CE0022908000E4936006E412082B4016A37476
:1007DE0000B582F07400B583EB9080007CE87D0458
:1007EE00DC04DD02D3227420A2AF92D1C2AFF0F0AE
:1007FE007B147AE5DAFEDBFA74A0F07A05DAFEE411
:10080E0093A2D192AFF470D8A37400B583EA7400AA
:10081E00B582E574FF908000F0E4F0C322F5F0EAB3
:10082E00C0E0EBC0E07A197440A2AF92D1C2AFF033
:10083E00E5F0F07B13DBFE74C0F07B05DBFEE4938A
:10084E00A2D192AFC395F06003DADCD3E4F0D0E02E
:10085E00FBD0E0FAE5F022C0E0C0F0F5F0740060E5
:10086E001BE583B4FF02800B5012B480028004504B
:10087E00028009E5F0112BD0F0D0E022E5F0F0E493
:10088E0093C395F06009E0C395F06003D38001C374
:10089E00D0F0D0E02232E4F5A8F5B875D00011A35F
:1008AE0011A3F4F580F590F5A0F5B075813079C8F7
:1008BE007AF9DAFED9FA7400601374B5600F78FA1B
:1008CE00A2B579C8D9FE4005D8F61207B675F0F96B
:1008DE0011F1311E75F0FD11F112007D7E007F8049
:1008EE000201DF90100012078C5024758204E493ED
:1008FE00B5F015C0F0C0837412C0E07409C0E07585
:10090E008240E473D083D0F00583E583B400D72210
:10091E0074007014E57B637A556379CC63781DB5EA
:10092E007A08B57905B5780221E475878075984205
:10093E00758911E4F588F58AF58CF58BF58D78C8F7
:10094E00791E30B0E5D9FBD8F720B0FD20B0FA20E3
:10095E00B0F720B0F420B0F130B0FDD28E208FCAA7
:10096E0020B0FA208FC430B0FA208FBE20B0FAD259
:10097E008C208FB630B0FAC28EC28C208FACE58B35
:10098E0033F5F0E58D3340A2A2F73400F404609AFB
:10099E00F58D758BFF758921D29CD28EE58DF40471
:1009AE00F978FFD8FED9FA309811C298E599547F9C
:1009BE0024F6600724056003020938E58A33F8E55A
:1009CE008C33F940F3E833F5F0E933A2F7340060E5
:1009DE00E7F404B58DE2F57BF57AF579F578637A6F
:1009EE00556379CC63781DF58DF58B7589217587E7
:1009FE0080759852D28E22309806120067B41B5121
:100A0E00120067B41B4B5173209803741B22120003
:100A1E0067B45B4451733098DE120067B4410374BF
:100A2E000B22B44203740A22B44303741522B44455
:100A3E0003740822B435028007B43602800280188F
:100A4E00C0E0517330980B120067B47E09D0E024D9
:100A5E00E422D0E080A1D0E0517330989A12006762
:100A6E00B41BF580A1EAC0E07A14E58C2098050449
:100A7E0070FADAF6D0E0FA22C0F0C0E08013C0F0CF
:100A8E00C0E030E70C742D120073D0E0C0E0F42407
:100A9E000175F06484D2D56007C2D524301200737C
:100AAE00E5F075F00A8430D502600524301200732B
:100ABE00E5F02430120073D0E0D0F022C0E0E8C0A0
:100ACE00E0C2D5AA82AB837C107D277128600724F3
:100ADE0030120073D2D57CE87D037128700330D5B7
:100AEE00072430120073D2D57C647D007128700308
:100AFE0030D5072430120073D2D5EAABF075F00A68
:100B0E0084700330D5052430120073E5F08BF02489
:100B1E0030120073D0E0F8D0E022780008C3EA9CCF
:100B2E00FAEB9DFB50F618EA2CFAEB3DFBE822C0DF
:100B3E00E0E8C0E0E9C0E0ECC0E0D2D1D2D5E49369
:100B4E00A3602520E72E547FB40D0712007DD2D16D
:100B5E0080ECB41F04C2D580E5B40E0512007D8072
:100B6E0007C2D112007380D6D0E0FCD0E0F9D0E0FD
:100B7E00F8D0E022547FF820D103120071C2D1C008
:100B8E0082C083900BF77C00E86007F971E670FC79
:100B9E00D9FA71E6603CB40F1271E60483801E68C8
:100BAE00667767796278766B716A7A0483800E65F0
:100BBE007461726E69736F6C756D706463A2D59299
:100BCE00E5D2D5B81402C2E5B80C02C2E512007324
:100BDE0080C0D083D082614CE493BC00057CFF546E
:100BEE000F227C00A3C4540F228290E82386054C6A
:100BFE00F844B3B0B1485FF0117FA0157F1C2ED121
:100C0E00405A50F103BFBA0C2F96018D3F95380D07
:100C1E006F5F1207710E562F483B6258201F767079
:100C2E00322440B840E1618F01340BCA89D3C0A38E
:100C3E00B9588004F80285602591F092731F107FD9
:100C4E0012549310444807D126564FD0F66472E0E2
:100C5E00B83BD5F0164F56306F48025FA8201F01E3
:100C6E007630D5602541A42C60056F013F261F30DC
:100C7E00078E1DF06399F042B8201F2330027AD1FF
:100C8E00602FF0F6058F931A5028F082046FA30D93
:100C9E003F1F514023013E0543017A0117649330F3
:100CAE002A088C243099B0F31960254135098ECB72
:100CBE00191230051F311D04144F761204AB279004
:100CCE0056012FA8D5F0AA26205F1CF0F361FE0175
:100CDE0041730127C1C0848FD6018770564F19709A
:100CEE001FA8D99076021743FE01C1840B157F020F
:100CFE008B14308F63396F19F011C9106D023F914B
:100D0E00097A41D0BA0C1D395F07F2111720416BD9
:100D1E003509F775120BA7CC48023F6412A00C27B9
:100D2E00E39FC014777011407121C0682541F062B5
:100D3E007FD1D021E16258B0F3051F733077B16FC8
:100D4E0019E01943E0582FF6A414D02303FE31F511
:100D5E00143099F8033F6422516025412FE3015668
:100D6E00279309FE11FE79BA607542EA6258A0E532
:100D7E001F534FD1C0A3094253F71204621B30F523
:100D8E0005F7690C351B70822F2F144F51C0642547
:100D9E000057656C636F6D658094322C2062791FED
:100DAE00F81FFE0D0E202053656594322E444F43DE
:100DBE002C94322E455155A494322E484452B4D51B
:100DCE008D2E0E201F9E1FA0210D0E9432204C6FD3
:100DDE00633A00203EA086CA822800292C958C807A
:100DEE00C83A20001F9782C373C7A6832CBA204A25
:100DFE00554D508086A172820D0E0D0D1F87838179
:100E0E003A20001FE4FB206B65793A20000D0D1F80
:100E1E00888083812028000D0D1F821FFD001F81F9
:100E2E0020202020201FC90E29201F871FB23A2004
:100E3E000046697273741F813A20004C6173741FEF
:100E4E00813A2020001FB9A120737572653F000DF5
:100E5E000D1F9C9A922C8C80C80E20201F9CC12C9A
:100E6E008E81F70D0E0D0D1F9F206173636969F959
:100E7E00961F9884892C958C80A00D0E0D1F8AA02C
:100E8E0065640D0E0D1F8AC1640D0E53756D6D6177
:100E9E0072793A0E20C67391640E208B91640E20E7
:100EAE008B207772697474656E0E1F9B3A0E208BC1
:100EBE0020756E61626C65802077726974650E2094
:100ECE0020626164F5730E20859F96C60E20858480
:100EDE009D0E2085206E6F6E849D0E1F979B206445
:100EEE00657465637465640D0E0D866E696E67823A
:100EFE003A0D0E0D0D53656E64696E671F988489E9
:100F0E00AC20200020802020000D0D5374616E64F3
:100F1E006172641F9E730E1FDA1FF465641F9E7349
:100F2E000E1F9A9E001F82001F8F1FE21FAA003FF6
:100F3E003F3F001FD7001F8ED7D1001FD1827300F5
:100F4E001F8682001F8A001F93001F8781001F8843
:100F5E00808381001F84DB9A83001F84DBC08300A3
:100F6E001F9C9A92001FED83001FCB9990001F9932
:0A0F7E0090CB640D0E1F859B0D0E35
:10100000A5E5E0A5FE4C0000000000000000000087
:10101000000000000000000000000000FFFFFFFFD4
:081020004C69737400020048E2
:1010400011257D14C2D1114CDDFC0125EFF5835132
:101050004FEEF582514FE493FAA3E493FBA3E4939C
:10106000FCEA5408700FEA035478F8EA54074890F1
:1010700016C8938008EAC4540F901362935403F87F
:101080002EFEEF3400FF743A512A719D20D121EADF
:10109000514F719DB80104790B8011EB514F719D37
:1010A000B8020479088005EC514F7906719DD9FC8E
:1010B000EA54087010901748EA035478F8EA540785
:1010C0004893F980099017C8EAC4540F93F9901B0C
:1010D0003E7808C374204007E99309A2E7547F5182
:1010E0002AD8F1741BC0E07411C0E0EA5408700FF4
:1010F000EA035478F8EA5407489016C8938008EA3F
:10110000C4540F9013629354FC03031490111D23D5
:101110002582F582E43583F583E4730125412D4171
:101120003C21812172414841044152415821A22170
:10113000D7415E4169416D4108411021AA218321B7
:101140007441714177417D413E411C418121DF4124
:101150001441C54185418B41914195419B41A94134
:10116000AF41B541BB410C41BF41CB41D741E74104
:10117000ED2231F67440512A7452512AEA54014149
:101180004531F6EB20E703EB414F9012F5E493A3D2
:1011900060F5F8C39B7003020038E493A330E7FACC
:1011A00080EB511031F8742F512AEB547823C4F896
:1011B000EB54806014901372E893901BD33582F542
:1011C000825002058331978005E82420514F742E08
:1011D000512AEB5407414531F6318331F8ECFBEBF2
:1011E0002EF582EB20E703E48002E4F43FF583026E
:1011F00000367440412A5108742C512A7420412A27
:101200007423412A318331F87441412A31AA31F8DB
:101210007443412A31F25108742B512A7444512AE3
:101220007450512A7454512A7452020030EF54F809
:10123000F8EAC403540748514FEB414F31F674525A
:10124000512AEA540702002E510831F85100EB02EE
:1012500000343183ECFB414A511031F821AA510886
:1012600031F85100EB514F21DB513E416031744167
:101270006051087442412A513E31F821DF31832107
:10128000DB31AA21DB513E31F84108513E31F821D2
:1012900083513E414A318331F8413EEBC0E0ECFBE3
:1012A000318331F8D0E0FB2183318331F82174316F
:1012B0007431F84108317431F821833174414A5155
:1012C0001C31F85100EB514FEC414F31F631F251E6
:1012D00008742B512A411C31F631F25108742B51FC
:1012E0002A7450512A411031F631F2411C31F25129
:1012F0001C31F84108E04143C38153D0824450CCB3
:10130000834450C88050B09050B1A050B2B050B398
:1013100099534255C6CD5448B2C85432434FCECCEF
:10132000544CB2CB5243415032C8CA52434150325E
:10133000CC8C5448B08A544CB08D5448B18B544C2A
:10134000B1F0C2D05053D7A849C5B849D089544D3F
:101350004FC48854434FCE9853434FCE8750434F8A
:10136000CE00595909090909097A7E0976330952CB
:101370000971000206080C0E101214161B1E202301
:101380002425F8F0E493C398227950E58DF404F80D
:10139000D8FED9F722514F743A412A514F74204157
:0113A0002A22
:10140000A5E5E0A5FE53000000000000000000007C
:10141000000000000000000000000000FFFFFFFFD0
:0C14200053696E676C652D537465700095
:1014400030B3069019C5020045900013E49324FEC2
:1014500060059019E88146A393F8E4A393F5828888
:101460008374027182700EA3741471827007A37466
:10147000EF71826011A882A9839019F59146E95114
:101480004FE8514F0125E5B85404F5B89019A891DB
:1014900046EF514FEE514F901992914612003C2069
:1014A000D50D50079019B131970125AE82AF83C297
:1014B0008A901A049146901AFC3197E4758108C00D
:1014C000E0C0E08E828F83F5D0F8F9FAFBFCFDFED8
:1014D000FFF5F0757CDD757D14D2AAD2AF737189EA
:1014E000D0E0F9D0E0F8D082D083D0D0D0E032C0C4
:1014F000E0C0D0C083C082E8C0E0E9C0E07189D21A
:1015000099719D719DE58124FBF8E6719BE5F07171
:101510009B08E62354015145719D08E6514F08E6AA
:10152000719B719D08E6719508E67195EA7195EBDE
:101530007195EC7195ED7195EE7195EF719B719DC3
:10154000E824F8719B719D719DE57C8E7CFEE57DA4
:101550008F7DFFEAC0E0EBC0E0ECC0E0D2D1114CDF
:10156000D0E0FCD0E0FBD0E0FAAF7DAE7CE581249A
:10157000F9F8E6F57C08E6F57D120062120040B449
:101580000D0281DEB4200281DEB43F07901A75910E
:1015900046A179B45113901AF53197C2AA71897591
:1015A000080075090075810932B44802A1CDB45212
:1015B00002A1FDB45302C167B44102C1AAB42E070F
:1015C000901AFC3197A179A179743D412A901A4370
:1015D0003197E47195719DA88118E6719B08E651D9
:1015E0004F7802790EA1ECE871957910719DE65162
:1015F0004F08D9F81125B880EE1125A17990134430
:101600003197B1C9E58124FCF8E6719B901348A895
:10161000A8D16090134BA8B8D16090134EA889D17F
:1016200060901353A888D160901358A898D1609007
:10163000135DA887D1607454512A7430512AB1C9FE
:10164000E58C514FE58A514F719D7454512A743184
:10165000512AB1C9E58D514FE58B514F1125A17923
:101660003197B1C9E8619B7817719DD8FC901A2B0E
:101670003197E58124F9F8E68E7CFE08E68F7DFF40
:10168000EAC0E0EBC0E0ECC0E0D2D1114CD0E0FC0D
:10169000D0E0FBD0E0FAE58124F9F8EEAE7CF57CF1
:1016A000F608EFAF7DF57DF6A179E58124FBF89092
:1016B0001A65319712003A400820D505F61125A188
:1016C000799019B13197A179AD066F3939464949F9
:1016D00063066F39394649496306AD39160E111153
:1016E0006306AD39160E111166061A1F160E11117A
:1016F00066061A1F160E111166061A1F160E111114
:1017000066062269161F9292660622A14D8386867E
:101710009B06969D160E11112606225D4DAD8E8EEE
:101720002606423D2F2B37374606423D390E111112
:101730004606423D39571111A5061111390E1111F6
:10174000A9068989391A89895A0E48732B2B2B2BA4
:1017500030004375212121212E0E676E06060606F4
:1017600038006A700A0A0A0A330E5D5D5D5D5D5DD0
:101770003B00121212121212410E8F8F8F8F8F8F19
:101780003E005D354C4C4C4C7C0E124F244C4C4C66
:101790004C004C4F808080805D0E4C2B57924C4CFF
:1017A00012001C1C15151515630E191984888888DC
:1017B000600078781F278B8B530E5353194C4C4C79
:1017C000530053531C4C4C4C2B21060A5D128F4C7A
:0817D0004C804C1588274C4C9D
:10180000A5E5E0A5FE41000000000000000000008A
:10181000000000000000000000000000FFFFFFFFCC
:0F18200041626F7574205041554C4D4F4E320050
:101840009018491200380210250D0A205041554CBD
:101850004D4F4E32206279205061756C2053746F69
:101860006666726567656E207061756C406563655C
:101870002E6F7273742E6564750D0A206D6F646926
:1018800066696564206279205769636869742053CA
:1018900069726963686F7465204A756C79203235A6
:1018A0002C2739390D0A202A20616464207265745E
:1018B00075726E207061746820746F206D6F6E6930
:1018C000746F722026207072696E74204143432029
:1018D00026205053570D0A202A207573652039366B
:1018E00030302066697865642062617564207261B9
:0518F00074650D0A0003
:10190000A5E5E0A5F9FF00000000000000000000D0
:10191000000000000000000000000000FFFFFFFFCB
:10192000466978656420426175642052617465007F
:1019400074FAF57BF57AF579F578637A556379CC95
:1019500063781D22C0D0C0E012004890197C1200AC
:1019600038D0E012003412004890198B120038D0A1
:10197000D0E5D012003412004802000041636375C4
:101980006D756C61746F72203D2000505357203D7F
:101990002000292C206F72203C4553433E20746F59
:1019A00020657869743A20000D1F88808381202883
:1019B0000020436F6D6D616E642041626F727465CB
:1019C000642E0D0A000DA1C520636F6E6E656374F1
:1019D00020494E5431202870696E20313329206C03
:1019E0006F7780BACFCC0D009432B3C7AE81203070
:1019F0003031330D001FB8B3FFA520766563746FD7
:101A000072AE20000D4E6F77866E696E67A6CFCCE2
:101A1000206D6F64653A20203C5245543E3DCC2CED
:101A2000203F3D2048656C700D0D00536B69707050
:101A3000696E6720496E737472756374696F6E2D79
:101A40003E20000D0A4C6F633A2020496E742052EC
:101A5000414D204D656D6F727920436F6E74656ED8
:101A600074730D0A004E6577204163632056616CE4
:101A700075653A20000D1FCF1FCC1F9E3A0D3C52BA
:101A800045543E2086D4F60D203C53503E2086D44B
:101A9000F60D20273F272020FF8ED70D20272E2749
:101AA0002020FFC4FD730D202752272020FF207324
:101AB00070656369616C2066756E6374696F6EC46E
:101AC000730D20274827202084DBC0920D20275348
:101AD000272020FCD4F60D202741272020F0A2202B
:101AE0004163632076616C75650D202751272020A6
:101AF000C8CFCC0D0E517569740D0A0020204143EA
:101B0000432042204320445054522020523020523F
:101B10003120523220523320523420523520523656
:101B2000205237202053502020204164647220200E
:101B3000496E737472756374696F6E0D0A00414368
:101B4000414CCC004144C400414444C3414A4DD0BF
:101B5000414ECC434A4EC5434CD24350CC44C14481
:101B600045C34449D6444A4EDA494EC34AC24A4262
:101B7000C34AC34A4DD04A4EC24A4EC34A4EDA4ABD
:101B8000DA4C43414CCC4C4A4DD04D4FD64D4F567C
:101B9000C34D4F56D84D55CC4E4FD04F52CC504FD1
:101BA000D0505553C85245D4524554C952CC524CCA
:101BB000C352D25252C3534554C2534A4DD05355C7
:101BC00042C2535741D05843C8584348C45852CCD6
:101BD0003F3FBF50B054434FCE50B153434FCE5010
:101BE000B249C550B349D043B05432434FCE50539D
:091BF000D744B84143C3FDC2FE15
:00000001FF
